:1000000057C071C05BC26FC06EC06DC06CC06BC0AA
:100010006AC069C068C067C066C065C064C063C0AC
:1000200062C005010905A1010901A10009300931DA
:1000300015002502750295028102C00509190129E2
:100040000415002501750195048102C0040309040B
:100050001C034200690064006F00750069006C00B9
:100060006C0065002E006F007200670010034E00E8
:10007000450053002000500061006400120110018F
:1000800000000008C016EB03000101020001090294
:100090002200010100803209040000010300000079
:1000A000092101010001222A000705810308000A35
:1000B00011241FBECFE5D1E0DEBFCDBF10E0A0E62A
:1000C000B0E0E4E3F7E002C005900D92A236B1077C
:1000D000D9F710E0A2E6B0E001C01D92AA39B1073D
:1000E000E1F704D025C38CCF80E00895FF920F93F1
:1000F0001F9380E395E70197F1F7479A92D0D09A42
:1001000080E197E22CE231E0F9013197F1F70197B4
:10011000D9F7D0987894D39AD298D79ADB98DF9869
:1001200085E0F82E14E005E287D080916F0084FF0F
:10013000FBCFF0926300DF9A812F8A95F1F7DF9869
:10014000812F8A95F1F7CA9902C000936300DB9A68
:10015000812F8A95F1F7CA9905C08091630080616B
:1001600080936300DB9A812F8A95F1F7CA9905C0C5
:1001700080916300806480936300DB9A812F8A956D
:10018000F1F7CA9905C0809163008068809363008D
:10019000DB9A812F8A95F1F7CA990DC0909163007F
:1001A000892F869586958D5F8370880F880F937F42
:1001B000982B90936300DB9A812F8A95F1F7CA9967
:1001C0000DC090916300892F869586958F5F83700F
:1001D000880F880F937F982B90936300DB9A812F71
:1001E0008A95F1F7CA9909C080916300982F9D5FA5
:1001F00093708C7F892B80936300DB9A812F8A9583
:10020000F1F7CA9909C080916300982F9F5F93709E
:100210008C7F892B8093630083E690E061E014D1AA
:1002200083CF919A8BB780618BBF8BE480937000F2
:100230008AE580936F0008951F93CF93DF93909189
:100240008000935097FDA5C020917D0080917C0097
:100250008D3209F09CC0983009F099C0CCE0D0E014
:10026000C21BD109CC57DF4F83EC809364008AE531
:1002700080936000109262008881807621F0CE0128
:1002800033DF282F7BC09A8110926D0089818823EB
:1002900021F410926E0022E06BC0853019F4909327
:1002A000810065C0863009F04EC08B81813041F4F9
:1002B0008CE790E090937F0080937E0022E13FC026
:1002C000823041F48EE890E090937F0080937E002E
:1002D00022E235C08330F1F4992341F48CE490E0BC
:1002E00090937F0080937E0024E029C0913041F4F8
:1002F00080E590E090937F0080937E002CE11FC00A
:100300009230E1F48CE690E090937F0080937E0041
:1003100020E115C0813241F480EA90E090937F00A3
:1003200080937E0029E00BC0823241F482E290E0AB
:1003300090937F0080937E002AE201C020E080E459
:10034000809362001BC0883021F421E083E890E0B4
:1003500011C0893019F49093830009C08A3011F4D8
:1003600021E006C08B3019F48BE48093700020E00C
:100370008DE690E090937F0080937E008F818823AC
:1003800021F48E81821708F4282F209361001092A7
:1003900080008091600084FF49C0809161008F3FA0
:1003A00009F444C0182F893008F018E0811B8093AD
:1003B00061008091640098E889278093640011238C
:1003C00041F120917E0030917F008091620086FF94
:1003D0000DC0A5E6B0E080E090E0F901E80FF91F5C
:1003E000E491ED9301961817C1F708C0912FD90138
:1003F000E5E6F0E08D9181939150E1F71150812F66
:1004000090E01F5F0196820F931F90937F0080936F
:100410007E0085E690E0612F4DD0612F6C5F6C30DF
:1004200019F08FEF809361006093600094E189B3CD
:10043000837031F49150D9F71092810010927B00B3
:10044000DF91CF911F9108951F93DC01162F8091AA
:100450006F0084FF07C08091700098E8892780931F
:10046000700003C08AE580936F00912FE1E7F0E010
:100470008D9181939150E1F781E790E0612F1AD03F
:100480001C5F10936F001F910895A82FB92F80E073
:1004900090E041E050EA609530E009C02D9182275C
:1004A0009795879510F084279527305EC8F36F5F86
:1004B000A8F30895EADF8D939D930895CF93CFB766
:1004C000CF93C395C89BE9F7C89B09C0C89B07C0D9
:1004D000C89B05C0C89B03C0C89B01C0A3C0DF93D5
:1004E000C0917D00DD27CC57DF4FC89B02C0DF9154
:1004F000EBCF2F930F931F9309B32FEF00FB20F93E
:100500004F933F9319B34FEF012700FB21F93BE0D5
:1005100031C04E7F012F19B3216028C0102F4D7FAD
:100520002260000009B329C04B7F2460012F000026
:1005300019B32BC019B3477F28602AC04F7E09B377
:1005400020612CC04F7D19B320622FC04F7B09B3AF
:10055000206432C0422709B349934FEF00001027AF
:1005600010FB20F919B31370C9F1297F91F201270B
:1005700000FB21F909B3237F89F2315058F110278C
:1005800010FB22F919B3277E79F2012700FB23F92A
:100590002F7C81F209B3102710FB24F92F7971F217
:1005A00000C019B3012700FB25F92F7359F200C0D1
:1005B00009B3102710FB26F9223040F200C019B30E
:1005C000012700FB27F9243028F64F77206819B35C
:1005D0000000F9CF10E11ABF002719C03B50319538
:1005E000C31BD04010E11ABF0881033CF9F00B3463
:1005F000E9F020917B001981110F1213EDCF4A8190
:10060000441F093641F10D3211F0013E29F70093E4
:1006100082003F914F911F910F912F91DF91CAB7A7
:10062000C4FD4FCFCF91CFBFCF91189520918200BD
:10063000222379F310918000112369F534306AF197
:100640003093800020937C0010917D003BE0311BB3
:1006500030937D0022C0009180000130E4F40AE56F
:100660004F7049F43091600034FD19C00093600070
:10067000C4E6D0E018C030916F0034FD10C0009384
:100680006F00C0E7D0E00FC02795A8F45150A9F43F
:10069000220F0000F9CF4AE503C042ED01C0432F0D
:1006A000C4E1D0E032E01AB31360D89A1ABB0BB39E
:1006B00020E413E05F93012756E00BBB279520F45D
:1006C000515021F4220FF9CF012756E000003B5A88
:1006D0000BBBD0F2279528F4515029F4220F0000CB
:1006E000F9CF012756E027950BBB20F4515021F498
:1006F000220FF9CF012756E0299133230BBB21F6B6
:100700000C7F10918100110FC651D0400BBB11F02E
:1007100010937B0010E11ABF01601AB31C7F402FB9
:100720004C7F5F9100C000C00BBB1ABB4BBB71CFAD
:04073000F894FFCF6B
:020734005AFF6A
:00000001FF
